:020000040800F2
:1000000000060020E1020008E3020008E302000805
:10001000E3020008E3020008E3020008E30200082C
:10002000E3020008E3020008E3020008C930000808
:10003000E3020008E3020008E3020008E30200080C
:10004000E3020008E3020008E3020008E3020008FC
:10005000E3020008E30200082948000855480008A8
:1000600081480008AD480008D94800085911000827
:1000700081110008AD110008D9110008051200080F
:100080002D12000859120008E3020008E3020008DC
:10009000E3020008E3020008E30200080549000843
:1000A000E3020008E3020008E3020008E30200089C
:1000B000E3020008E3020008E3020008E30200088C
:1000C000E3020008E3020008E3020008E30200087C
:1000D000E3020008DD490008E3020008E30200082B
:1000E00069490008E3020008E3020008E30200088F
:1000F000E3020008E3020008E3020008851200089A
:10010000E3020008E3020008F1490008E3020008E6
:10011000E3020008E3020008E3020008E30200082B
:10012000B1120008D91200080513000831130008A5
:100130005D130008E3020008E3020008E302000880
:10014000E3020008E3020008E3020008E3020008FB
:1001500085130008B1130008DD130008E30200084E
:10016000E3020008E3020008E3020008E3020008DB
:10017000E3020008B53C0008E3020008E3020008BF
:10018000E3020008E3020008E3020008E3020008BB
:10019000E3020008E3020008E3020008E3020008AB
:1001A000E3020008E3020008E3020008E30200089B
:1001B000E3020008E3020008E3020008E30200088B
:1001C000E3020008E3020008E3020008E30200087B
:1001D000E3020008A13C0008E3020008E302000873
:1001E000E3020008E3020008E3020008E30200085B
:1001F000E3020008E3020008E3020008E30200084B
:10020000E3020008E3020008E3020008E30200083A
:10021000E3020008E3020008E3020008E30200082A
:10022000E3020008E3020008E3020008E30200081A
:10023000E3020008E3020008E3020008E30200080A
:10024000E3020008E3020008E3020008E3020008FA
:10025000E3020008E3020008E3020008E3020008EA
:10026000E3020008E3020008E3020008E3020008DA
:10027000E3020008E3020008E3020008E3020008CA
:10028000E3020008E3020008E3020008E3020008BA
:10029000E3020008E3020008E3020008E3020008AA
:1002A000E3020008E3020008E3020008E30200089A
:1002B000E3020008E3020008E3020008E30200088A
:1002C000E3020008E3020008E3020008E30200087A
:1002D000E3020008E3020008E3020008E30200086A
:1002E00002E000F000F8FEE772B6374880F30888B5
:1002F000364880F3098836483649086040F20000E5
:10030000CCF200004EF63471CEF200010860BFF36B
:100310004F8FBFF36F8F40F20000C0F2F0004EF637
:100320008851CEF200010860BFF34F8FBFF36F8F8B
:100330004FF00000E1EE100A4EF63C71CEF20001E3
:100340000860062080F31488BFF36F8F02F01EFF51
:1003500004F024F84FF055301F491B4A91423CBF2E
:1003600041F8040BFAE71D49184A91423CBF41F895
:10037000040BFAE71A491B4A1B4B9A423EBF51F83D
:10038000040B42F8040BF8E700201849184A914280
:100390003CBF41F8040BFAE702F036FF04F082F8A4
:1003A000144C154DAC4203DA54F8041B8847F9E7A6
:1003B00000F042F8114C124DAC4203DA54F8041B21
:1003C0008847F9E702F01EBF000600200022002047
:1003D0000000000808ED00E00000002000060020FA
:1003E000604F0008002200206422002068220020C4
:1003F0000C490020E0020008E0020008E0020008CA
:10040000E00200082DE9F04F2DED108AC1F80CD064
:10041000D0F80CD0BDEC108ABDE8F08F002383F338
:1004200011882846A047002002F014F9FEE702F0E8
:100430009FF800DFFEE7000038B500F045FC00F053
:1004400015FE02F001FE054602F034FE0446C0B976
:100450000E4B9D4217D001339D4241F2883512BFA9
:10046000044600250124002002F0F8FD0CB100F044
:1004700075F800F099FD284600F01EF900F06EF8BE
:10048000F9E70025EFE70546EDE700BF010007B0FB
:1004900008B500F0E5FBA0F120035842584108BD23
:1004A00007B541F21203022101A8ADF8043000F0B3
:1004B000F5FB03B05DF804FB38B5302383F31188F6
:1004C000174803680BB102F091F90023154A4FF465
:1004D0007A71134802F080F9002383F31188124CDB
:1004E000236813B12368013B2360636813B1636819
:1004F000013B63600D4D2B7833B963687BB90220F3
:1005000000F0B4FC322363602B78032B07D16368BF
:100510002BB9022000F0AAFC4FF47A73636038BD57
:1005200068220020B90400088823002080220020CF
:10053000084B187003280CD8DFE800F00805020803
:10054000022000F085BC022000F072BC024B0022A9
:100550005A6070478022002088230020F8B5504B55
:10056000504A1C461968013100F0998004339342C7
:10057000F8D162684C4B9A4240F291804B4B9B6899
:1005800003F1006303F500339A4280F08880002075
:1005900000F0C0FB0220FFF7CBFF454B0021D3F852
:1005A000E820C3F8E810D3F81021C3F81011D3F8ED
:1005B0001021D3F8EC20C3F8EC10D3F81421C3F8C1
:1005C0001411D3F81421D3F8F020C3F8F010D3F8A5
:1005D0001821C3F81811D3F81821D3F8802042F05D
:1005E0000062C3F88020D3F8802022F00062C3F8B4
:1005F0008020D3F88020D3F8802042F00072C3F826
:100600008020D3F8802022F00072C3F88020D3F835
:10061000803072B64FF0E023C3F8084DD4E90004EF
:10062000BFF34F8FBFF36F8F224AC2F88410BFF31E
:100630004F8F536923F480335361BFF34F8FD2F848
:10064000803043F6E076C3F3C905C3F34E335B0154
:1006500003EA060C29464CEA81770139C2F8747224
:10066000F9D2203B13F1200FF2D1BFF34F8FBFF32C
:100670006F8FBFF34F8FBFF36F8F536923F4003336
:1006800053610023C2F85032BFF34F8FBFF36F8F17
:10069000302383F31188854680F308882047F8BD0E
:1006A0000000020820000208FFFF010800220020CD
:1006B0000044025800ED00E02DE9F04F93B0B44B38
:1006C0002022FF2100900AA89D6800F017FCB14A83
:1006D0001378A3B90121B04811700360302383F36C
:1006E000118803680BB102F081F80023AB4A4FF484
:1006F0007A71A94802F070F8002383F31188009BF7
:1007000013B1A74B009A1A60A64A1378032B03D0A3
:1007100000231370A24A53604FF0000A009CD34696
:100720005646D146012000F093FB24B19C4B1B6838
:10073000002B00F02682002000F092FA0390039B29
:10074000002BF2DB012000F073FB039B213B1F2BEE
:10075000E8D801A252F823F0D907000801080008E0
:100760009508000825070008250700082507000848
:1007700027090008F70A0008110A0008730A000890
:100780009B0A0008C10A000825070008D30A0008D0
:1007900025070008450B0008790800082507000810
:1007A000890B0008E50700087908000825070008FC
:1007B000730A000825070008250700082507000818
:1007C0002507000825070008250700082507000859
:1007D00025070008950800080220FFF759FE0028A9
:1007E00040F0F981009B022105A8BAF1000F08BF73
:1007F0001C4641F21233ADF8143000F04FFA91E785
:100800004FF47A7000F02CFA071EEBDB0220FFF7A2
:100810003FFE0028E6D0013F052F00F2DE81DFE831
:1008200007F0030A0D1013360523042105A80593CC
:1008300000F034FA17E004215548F9E704215A483A
:10084000F6E704215948F3E74FF01C08404608F149
:10085000040800F061FA0421059005A800F01EFAD2
:10086000B8F12C0FF2D101204FF0000900FA07F780
:1008700047EA0B0B5FFA8BFB00F08CFB26B10BF009
:100880000B030B2B08BF0024FFF70AFE4AE70421E5
:100890004748CDE7002EA5D00BF00B030B2BA1D1C1
:1008A0000220FFF7F5FD074600289BD00120002617
:1008B00000F030FA0220FFF73BFE1FFA86F84046B0
:1008C00000F038FA0446B0B1039940460136A1F170
:1008D00040025142514100F03DFA0028EDD1BA46A4
:1008E000044641F21213022105A83E46ADF8143029
:1008F00000F0D4F916E725460120FFF719FE244B36
:100900009B68AB4207D9284600F006FA013040F058
:1009100067810435F3E70025224BBA463E461D7039
:100920001F4B5D60A8E7002E3FF45CAF0BF00B039C
:100930000B2B7FF457AF0220FFF7FAFD322000F0B7
:100940008FF9B0F10008FFF64DAF18F003077FF400
:1009500049AF0F4A08EB0503926893423FF642AF56
:10096000B8F5807F3FF73EAF124BB845019323DDCA
:100970004FF47A7000F074F90390039A002AFFF69E
:1009800031AF039A0137019B03F8012BEDE700BF5C
:10099000002200208423002068220020B9040008DF
:1009A000882300208022002004220020082200202A
:1009B0000C22002084220020C820FFF769FD074692
:1009C00000283FF40FAF1F2D11D8C5F120020AAB4C
:1009D00025F0030084494245184428BF424601924D
:1009E00000F066FA019AFF217F4800F087FA4FEA8B
:1009F000A803C8F387027C492846019300F086FAD1
:100A0000064600283FF46DAF019B05EB830533E7F5
:100A10000220FFF73DFD00283FF4E4AE00F0B8F9F6
:100A200000283FF4DFAE0027B846704B9B68BB42FE
:100A300018D91F2F11D80A9B01330ED027F00303BA
:100A400012AA134453F8203C05934046042205A9FA
:100A5000043700F06BFB8046E7E7384600F05CF9AE
:100A60000590F2E7CDF81480042105A800F016F9EE
:100A700002E70023642104A8049300F005F900288C
:100A80007FF4B0AE0220FFF703FD00283FF4AAAECA
:100A9000049800F073F90590E6E70023642104A8A8
:100AA000049300F0F1F800287FF49CAE0220FFF7D9
:100AB000EFFC00283FF496AE049800F061F9EAE7F5
:100AC0000220FFF7E5FC00283FF48CAE00F070F93F
:100AD000E1E70220FFF7DCFC00283FF483AE05A924
:100AE000142000F06BF907460421049004A800F0DC
:100AF000D5F83946B9E7322000F0B2F8071EFFF604
:100B000071AEBB077FF46EAE384A07EB09039268FB
:100B100093423FF667AE0220FFF7BAFC00283FF48D
:100B200061AE27F003074F44B9453FF4A5AE4846F0
:100B300009F1040900F0F0F80421059005A800F07F
:100B4000ADF8F1E74FF47A70FFF7A2FC00283FF40C
:100B500049AE00F01DF9002844D00A9B01330BD0A8
:100B600008220AA9002000F0D1F900283AD020225A
:100B7000FF210AA800F0C2F9FFF792FC1C4801F01F
:100B80006FFD13B0BDE8F08F002E3FF42BAE0BF0DD
:100B90000B030B2B7FF426AE0023642105A80593DD
:100BA00000F072F8074600287FF41CAE0220FFF721
:100BB0006FFC804600283FF415AEFFF771FC41F250
:100BC000883001F04DFD059800F02EFA46463C466F
:100BD00000F0E0F9A6E506464EE64FF0000901E612
:100BE000BA467EE637467CE68422002000220020BA
:100BF000A08601002DE9F84F4FF47A7306460D46A2
:100C0000002402FB03F7DFF85080DFF8509098F9DA
:100C100000305FFA84FA5A1C01D0A34212D159F86D
:100C200024002A4631460368D3F820B03B46D84713
:100C3000854207D1074B012083F800A0BDE8F88F5B
:100C40000124E4E7002CFBD04FF4FA7001F008FD1A
:100C50000020F3E7D42300201022002014220020DB
:100C6000002307B5024601210DF107008DF807307A
:100C7000FFF7C0FF20B19DF8070003B05DF804FB4B
:100C80004FF0FF30F9E700000A46042108B5FFF7EE
:100C9000B1FF80F00100C0B2404208BD074B0A46D8
:100CA00030B41978064B53F821400146236820469A
:100CB000DD69044BAC4630BC604700BFD423002044
:100CC00014220020A086010070B5104C0025104EA3
:100CD00001F0E4FF20803068238883420CD800258F
:100CE0002088013801F0D6FF23880544013BB5F583
:100CF000802F2380F4D370BD01F0CCFF336805440E
:100D00000133B5F5003F3360E5D3E8E7D623002093
:100D10009023002002F090B800F1006000F5003050
:100D20000068704700F10060920000F5003002F0AA
:100D300011B80000054B1A68054B1B889B1A8342AB
:100D400002D9104401F0A6BF002070479023002074
:100D5000D623002038B50446074D29B12868204421
:100D6000BDE8384001F0AEBF2868204401F098FF8C
:100D70000028F3D038BD00BF90230020002070472A
:100D800000F1FF5000F58F10D0F800087047000008
:100D9000064991F8243033B100230822086A81F80B
:100DA0002430FFF7BFBF0120704700BF942300200D
:100DB000014B1868704700BF0010005C194B0138E8
:100DC0000322084470B51D68174BC5F30B042D0CA6
:100DD0001E88A6420BD15C680A46013C824213463B
:100DE0000FD214F9016F4EB102F8016BF6E7013A28
:100DF00003F10803ECD181420B4602D22C2203F806
:100E0000012B0424094A1688AE4204D1984284BFBB
:100E1000967803F8016B013C02F10402F3D1581AF1
:100E200070BD00BF0010005C1C220020F44A0008C6
:100E3000022804D1054B4FF480129A6170470128B3
:100E4000FCD1024B4FF48022F7E700BF001002589C
:100E5000022803D1044B10229A6170470128FCD16B
:100E6000014B0422F8E700BF00100258022805D108
:100E7000064A536983F01003536170470128FCD17F
:100E8000024A536983F00403F6E700BF00100258DA
:100E900070B504464FF47A764CB1412C254628BFF4
:100EA000412506FB05F0641B01F0DAFBF4E770BD99
:100EB000002310B5934203D0CC5CC4540133F9E74E
:100EC00010BD0000013810B510F9013F3BB191F998
:100ED00000409C4203D11AB10131013AF4E71AB142
:100EE00091F90020981A10BD1046FCE7034602460F
:100EF000D01A12F9011B0029FAD1704702440346A7
:100F0000934202D003F8011BFAE770472DE9F8433A
:100F10001F4D14460746884695F8242052BBDFF83B
:100F200070909CB395F824302BB92022FF214846BD
:100F30002F62FFF7E3FF95F824004146C0F1080255
:100F400005EB8000A24228BF2246D6B29200FFF7EE
:100F5000AFFF95F82430A41B17441E449044E4B21C
:100F6000F6B2082E85F82460DBD1FFF711FF0028C8
:100F7000D7D108E02B6A03EB82038342CFD0FFF77F
:100F800007FF0028CBD10020BDE8F8830120FBE754
:100F900094230020024B1A78024B1A70704700BF4E
:100FA000D42300201022002038B51A4C1A4D2046B8
:100FB00000F086FE2946204600F0AEFE2D684FF474
:100FC0007A70D5F89020D2F8043843F00203C2F8C2
:100FD0000438FFF75DFF1149284600F0ABFFD5F854
:100FE00090200F4DD2F80438286823F002030D49F1
:100FF000A042C2F804384FF4E1330B6001D000F096
:10100000BDFD6868A04204D00649BDE8384000F044
:10101000B5BD38BD382B0020F04C0008F84C000856
:1010200014220020BC2300200C4B70B50C4D04464C
:101030001E780C4B55F826209A420DD00A4B002101
:1010400018221846FFF75AFF0460014655F826009B
:10105000BDE8704000F092BD70BD00BFD4230020F9
:1010600014220020382B0020BC230020F8B571B6D4
:10107000002301201A46194600F058FA0446802041
:1010800001F078FF002849D00025254A80274FF439
:10109000D06C3D26136913F0C06F26D1D2F8103101
:1010A00013F0C06F21D1236805F1006199602368B6
:1010B000D86023685F602368C3F800C021680B68AC
:1010C00043F001030B6021680B6823F01E030B60E3
:1010D00021680B68DB07FCD4237B8035616806FA46
:1010E00003F3B5F5001F0B60D4D1204600F05EFA83
:1010F000B5F5001F11D000240A4E0B4D012001F060
:101100009BFE3388A34205D928682044013401F0AE
:10111000D9FDF6E7002001F08FFE61B6F8BD00BFF3
:1011200000200052D62300209023002030B50A442E
:10113000084D91420DD011F8013B5840082340F36F
:101140000004013B2C4013F0FF0384EA5000F6D169
:10115000EFE730BD2083B8ED08B5074B074A1968A3
:1011600001F03D01996053680BB190689847BDE864
:10117000084001F0E1BF00BF00000240D82300207A
:1011800008B5084B1968890901F03D018A019A6088
:10119000054AD3680BB110699847BDE8084001F0D3
:1011A000CBBF00BF00000240D823002008B5084B89
:1011B0001968090C01F03D010A049A60054A536957
:1011C0000BB190699847BDE8084001F0B5BF00BF7A
:1011D00000000240D823002008B5084B1968890D8B
:1011E00001F03D018A059A60054AD3690BB1106A86
:1011F0009847BDE8084001F09FBF00BF00000240D3
:10120000D823002008B5074B074A596801F03D0173
:10121000D960536A0BB1906A9847BDE8084001F065
:101220008BBF00BF00000240D823002008B5084B48
:101230005968890901F03D018A01DA60054AD36ADB
:101240000BB1106B9847BDE8084001F075BF00BFB7
:1012500000000240D823002008B5084B5968090C4B
:1012600001F03D010A04DA60054A536B0BB1906B43
:101270009847BDE8084001F05FBF00BF0000024092
:10128000D823002008B5084B5968890D01F03D01AD
:101290008A05DA60054AD36B0BB1106C9847BDE83C
:1012A000084001F049BF00BF00000240D8230020E1
:1012B00008B5074B074A196801F03D019960536C66
:1012C0000BB1906C9847BDE8084001F035BF00BFF6
:1012D00000040240D823002008B5084B196889098A
:1012E00001F03D018A019A60054AD36C0BB1106D83
:1012F0009847BDE8084001F01FBF00BF000402404E
:10130000D823002008B5084B1968090C01F03D01ED
:101310000A049A60054A536D0BB1906D9847BDE879
:10132000084001F009BF00BF00040240D82300209C
:1013300008B5084B1968890D01F03D018A059A60CE
:10134000054AD36D0BB1106E9847BDE8084001F017
:10135000F3BE00BF00040240D823002008B5074BAD
:10136000074A596801F03D01D960536E0BB1906E88
:101370009847BDE8084001F0DFBE00BF000402400E
:10138000D823002008B5084B5968890901F03D01B0
:101390008A01DA60054AD36E0BB1106F9847BDE839
:1013A000084001F0C9BE00BF00040240D82300205D
:1013B00008B5084B5968090C01F03D010A04DA60D0
:1013C000054A536F0BB1906F9847BDE8084001F094
:1013D000B3BE00BF00040240D823002008B5084B6C
:1013E0005968890D01F03D018A05DA60054AD36F1D
:1013F00013B1D2F880009847BDE8084001F09CBEC8
:1014000000040240D823002000230C4910B51A46DE
:101410000B4C0B6054F82300026001EB43000433D3
:101420004260402BF6D1074A4FF0FF339360D36000
:10143000C2F80834C2F80C3410BD00BFD823002015
:10144000044B0008000002400F28F8B510D91028FE
:1014500010D0112811D0122808D10F240720DFF84E
:10146000C8E00126DEF80050A04208D9002653E06B
:101470000446F4E70F240020F1E70724FBE706FA0F
:1014800000F73D424AD1264C4FEA001C3D4304EB95
:1014900000160EEBC000CEF80050C0E90123FBB2ED
:1014A00073B12048D0F8D83043F00103C0F8D830E9
:1014B000D0F8003143F00103C0F80031D0F800311A
:1014C00017F47F4F0ED01748D0F8D83043F00203FE
:1014D000C0F8D830D0F8003143F00203C0F8003132
:1014E000D0F8003154F80C00036823F01F030360A8
:1014F000056815F00105FBD104EB0C033D2493F8BE
:101500000CC05F6804FA0CF43C602124056044615F
:1015100012B1987B00F066F93046F8BD0130A3E7C0
:10152000044B000800440258D823002010B5302492
:1015300084F31188FFF788FF002383F3118810BD1F
:1015400010B50446807B00F063F901231549627BE6
:1015500003FA02F20B6823EA0203DAB20B6072B9F3
:10156000114AD2F8D81021F00101C2F8D810D2F8EF
:10157000001121F00101C2F80011D2F8002113F48A
:101580007F4F0ED1084BD3F8D82022F00202C3F8C7
:10159000D820D3F8002122F00202C3F80021D3F8AA
:1015A000003110BDD82300200044025808B5302374
:1015B00083F31188FFF7C4FF002383F3118808BD6C
:1015C000026843681143016003B118477047000087
:1015D000024A136843F0C0031360704700100140D3
:1015E00013B50E4C204600F0BDFA04F114000023A0
:1015F0004FF400720A49009400F07AF9094B4FF455
:101600000072094904F13800009400F0F3F9074A28
:10161000074BC4E9172302B010BD00BF5C240020B3
:10162000C8240020D1150008C82600200010014061
:1016300000E1F505037C30B5244C002918BF0C46A9
:10164000012B11D1224B98420ED1224BD3F8F0201E
:1016500042F01002C3F8F020D3F8182142F0100233
:10166000C3F81821D3F818312268036EC16D03EB5B
:1016700052038466B3FBF2F36268150442BF23F0A1
:10168000070503F0070343EA4503CB60A36843F073
:1016900040034B60E36843F001038B6042F49673B0
:1016A00043F001030B604FF0FF330B62510505D58A
:1016B00012F0102205D0B2F1805F04D080F86430BF
:1016C00030BD7F23FAE73F23F8E700BF044C000852
:1016D0005C240020004402582DE9F047C66D054601
:1016E0003768F469210734621AD014F0080118BF72
:1016F0004FF48071E20748BF41F02001A3074FF08B
:10170000300348BF41F04001600748BF41F080010D
:1017100083F31188281DFFF753FF002383F31188FB
:10172000E2050AD5302383F311884FF48061281D28
:10173000FFF746FF002383F311884FF030094FF085
:10174000000A14F0200838D13B0616D54FF03009B6
:1017500005F1380A200610D589F31188504600F0AB
:101760007DF9002836DA0821281DFFF729FF27F028
:1017700080033360002383F31188790614D5620651
:1017800012D5302383F31188D5E913239A4208D167
:101790002B6C33B127F040071021281DFFF710FFF5
:1017A0003760002383F31188E30618D5AA6E136906
:1017B000ABB15069BDE8F047184789F31188736AE7
:1017C000284695F86410194000F0E6F98AF311886C
:1017D000F469B6E7B06288F31188F469BAE7BDE846
:1017E000F0870000090100F16043012203F5614325
:1017F000C9B283F8001300F01F039A4043099B000D
:1018000003F1604303F56143C3F880211A60704718
:1018100000F01F0301229A40430900F160409B0041
:1018200000F5614003F1604303F56143C3F8802094
:10183000C3F88021002380F800337047F8B51546BF
:10184000826804460B46AA4200D28568A1692669CF
:10185000761AB5420BD218462A46FFF729FBA36930
:101860002B44A3612846A3685B1BA360F8BD0CD979
:10187000AF1B18463246FFF71BFB3A46E16830447F
:10188000FFF716FBE3683B44EBE718462A46FFF7F1
:101890000FFBE368E5E7000083689342F7B5044671
:1018A000154600D28568D4E90460361AB5420BD2D9
:1018B0002A46FFF7FDFA63692B4463612846A36853
:1018C0005B1BA36003B0F0BD0DD93246AF1B019185
:1018D000FFF7EEFA01993A46E0683144FFF7E8FA7B
:1018E000E3683B44E9E72A46FFF7E2FAE368E4E706
:1018F00010B50A440024C361029B8460C160026188
:101900000362C0E90000C0E9051110BD08B5D0E9C7
:101910000532934201D1826882B9826801328260C5
:101920005A1C426119700021D0E904329A4224BF46
:10193000C368436100F0B0FE002008BD4FF0FF30E7
:10194000FBE7000070B5302304460E4683F3118890
:10195000A568A5B1A368A269013BA360531CA3615C
:1019600015782269934224BFE368A361E3690BB150
:1019700020469847002383F31188284607E0314624
:10198000204600F079FE0028E2DA85F3118870BD68
:101990002DE9F74F04460E4617469846D0F81C909E
:1019A0004FF0300A8AF311884FF0000B154665B1ED
:1019B0002A4631462046FFF741FF034660B94146BB
:1019C000204600F059FE0028F1D0002383F311884F
:1019D000781B03B0BDE8F08FB9F1000F03D0019080
:1019E0002046C847019B8BF31188ED1A1E448AF3E9
:1019F0001188DCE7C160C361009B82600362C0E9BB
:101A000005111144C0E9000001617047F8B50446B2
:101A10000D461646302383F31188A768A7B1A36843
:101A2000013BA36063695A1C62611D70D4E90432F2
:101A30009A4224BFE3686361E3690BB1204698478B
:101A4000002080F3118807E03146204600F014FEA4
:101A50000028E2DA87F31188F8BD0000D0E90523F9
:101A600010B59A4201D182687AB9826800210132A8
:101A700082605A1C82611C7803699A4224BFC36841
:101A8000836100F009FE204610BD4FF0FF30FBE7F8
:101A90002DE9F74F04460E4617469846D0F81C909D
:101AA0004FF0300A8AF311884FF0000B154665B1EC
:101AB0002A4631462046FFF7EFFE034660B941460D
:101AC000204600F0D9FD0028F1D0002383F31188CF
:101AD000781B03B0BDE8F08FB9F1000F03D001907F
:101AE0002046C847019B8BF31188ED1A1E448AF3E8
:101AF0001188DCE7026843681143016003B11847AD
:101B0000704700001430FFF743BF00004FF0FF3371
:101B10001430FFF73DBF00003830FFF7B9BF0000B9
:101B20004FF0FF333830FFF7B3BF00001430FFF73A
:101B300009BF00004FF0FF311430FFF703BF000072
:101B40003830FFF763BF00004FF0FF323830FFF747
:101B50005DBF0000012914BF6FF013000020704723
:101B6000FFF73EBD044B036000234360C0E902332E
:101B700001230374704700BF1C4C000810B53023CC
:101B8000044683F31188FFF755FD022300202374D8
:101B900080F3118810BD000038B5C36904460D46B6
:101BA0001BB904210844FFF7A5FF294604F11400DE
:101BB000FFF7ACFE002806DA201D4FF40061BDE8F7
:101BC0003840FFF797BF38BD026843681143016092
:101BD00003B118477047000013B5406B00F58054FF
:101BE000D4F8A4381A681178042914D1017C022988
:101BF00011D11979012312898B4013420BD101A90C
:101C00004C3002F089F9D4F8A4480246019B2179AE
:101C1000206800F0DFF902B010BD0000143002F0BF
:101C20000BB900004FF0FF33143002F005B900008B
:101C30004C3002F0DDB900004FF0FF334C3002F0C1
:101C4000D7B90000143002F0D9B800004FF0FF31CE
:101C5000143002F0D3B800004C3002F0A9B90000F3
:101C60004FF0FF324C3002F0A3B900000020704763
:101C700010B500F58054D4F8A4381A6811780429F6
:101C800017D1017C022914D15979012352898B4043
:101C900013420ED1143002F06BF8024648B1D4F86A
:101CA000A4484FF4407361792068BDE8104000F00B
:101CB0007FB910BD406BFFF7DBBF0000704700002D
:101CC0007FB5124B012504260446036000230574EA
:101CD00000F1840243602946C0E902330C4B0290B4
:101CE000143001934FF44073009602F01DF8094B35
:101CF00004F69442294604F14C000294CDE90063B5
:101D00004FF4407302F0E4F804B070BD444C000896
:101D1000B51C0008D91B00080A68302383F311881A
:101D20000B790B3342F823004B79133342F823002D
:101D30008B7913B10B3342F8230000F58053C3F8BD
:101D4000A41802230374002080F311887047000058
:101D500038B5037F044613B190F85430ABB9012570
:101D6000201D0221FFF730FF04F114006FF0010184
:101D7000257700F09DFC04F14C0084F854506FF07E
:101D80000101BDE8384000F093BC38BD10B5012119
:101D900004460430FFF718FF0023237784F85430FB
:101DA00010BD000038B504460025143001F0D4FF02
:101DB00004F14C00257702F0A3F8201D84F854505C
:101DC0000121FFF701FF2046BDE83840FFF750BF73
:101DD00090F8803003F06003202B06D190F881202A
:101DE0000023212A03D81F2A06D800207047222A60
:101DF000FBD1C0E91D3303E0034A42670722826733
:101E0000C3670120704700BF3422002037B500F5BA
:101E10008055D5F8A4381A68117804291AD1017CA4
:101E2000022917D11979012312898B40134211D14C
:101E300000F14C04204602F023F958B101A92046D4
:101E400002F06AF8D5F8A4480246019B217920687F
:101E500000F0C0F803B030BD01F10B03F0B550F84D
:101E6000236085B004460D46FEB1302383F311880C
:101E700004EB8507301D0821FFF7A6FEFB6806F17D
:101E80004C005B691B681BB1019002F053F801988C
:101E900003A902F041F8024648B1039B29462046B7
:101EA00000F098F8002383F3118805B0F0BDFB68BB
:101EB0005A691268002AF5D01B8A013B1340F1D100
:101EC00004F18002EAE70000133138B550F82140F0
:101ED000ECB1302383F3118804F58053D3F8A428A0
:101EE0001368527903EB8203DB689B695D6845B137
:101EF00004216018FFF768FE294604F1140001F080
:101F000041FF2046FFF7B4FE002383F3118838BD5C
:101F10007047000001F00EBA01234022002110B5E5
:101F2000044600F8303BFEF7E9FF0023C4E9013323
:101F300010BD000010B53023044683F3118824221D
:101F4000416000210C30FEF7D9FF204601F014FA61
:101F500002230020237080F3118810BD70B500EBC0
:101F60008103054650690E461446DA6018B1102206
:101F70000021FEF7C3FFA06918B110220021FEF76F
:101F8000BDFF31462846BDE8704001F0FBBA0000B5
:101F900083682022002103F0011310B504468360FA
:101FA0001030FEF7ABFF2046BDE8104001F076BBD5
:101FB000F0B4012500EB810447898D40E4683D437E
:101FC000A469458123600023A2606360F0BC01F036
:101FD00093BB0000F0B4012500EB810407898D401C
:101FE000E4683D436469058123600023A260636067
:101FF000F0BC01F009BC000070B5022300250446C6
:10200000242203702946C0F888500C3040F8045C44
:10201000FEF774FF204684F8705001F047FA6368B9
:102020001B6823B129462046BDE87040184770BDA3
:102030000378052B10B504460AD080F88C300523B0
:10204000037043681B680BB1042198470023A36009
:1020500010BD00000178052906D190F88C20436856
:1020600002701B6803B118477047000070B590F804
:102070007030044613B1002380F8703004F1800200
:10208000204601F02FFB63689B68B3B994F8803059
:1020900013F0600535D00021204601F021FE00211B
:1020A000204601F011FE63681B6813B1062120462B
:1020B0009847062384F8703070BD20469847002862
:1020C000E4D0B4F88630A26F9A4288BFA36794F92F
:1020D0008030A56F002B4FF0300380F20381002D7C
:1020E00000F0F280092284F8702083F31188002127
:1020F0002046D4E91D23FFF76DFF002383F31188E9
:10210000DAE794F8812003F07F0343EA022340F2E8
:102110000232934200F0C58021D8B3F5807F48D0C9
:102120000DD8012B3FD0022B00F09380002BB2D1B1
:1021300004F1880262670222A267E367C1E7B3F590
:10214000817F00F09B80B3F5407FA4D194F882306A
:10215000012BA0D1B4F8883043F0020332E0B3F58C
:10216000006F4DD017D8B3F5A06F31D0A3F5C06381
:10217000012B90D86368204694F882205E6894F81A
:102180008310B4F88430B047002884D04368636774
:102190000368A3671AE0B3F5106F36D040F6024229
:1021A00093427FF478AF5C4B63670223A3670023FD
:1021B000C3E794F88230012B7FF46DAFB4F8883018
:1021C00023F00203A4F88830C4E91D55E56778E7D9
:1021D000B4F88030B3F5A06F0ED194F88230204669
:1021E00084F88A3001F0C0F963681B6813B10121DB
:1021F00020469847032323700023C4E91D339CE73E
:1022000004F18B0363670123C3E72378042B10D108
:10221000302383F311882046FFF7BAFE85F3118837
:102220000321636884F88B5021701B680BB1204632
:10223000984794F88230002BDED084F88B3004234A
:10224000237063681B68002BD6D002212046984774
:10225000D2E794F8843020461D0603F00F010AD51A
:1022600001F032FA012804D002287FF414AF2B4B7E
:102270009AE72B4B98E701F019FAF3E794F88230CC
:10228000002B7FF408AF94F8843013F00F01B3D023
:102290001A06204602D501F03BFDADE701F02CFD0A
:1022A000AAE794F88230002B7FF4F5AE94F88430DE
:1022B00013F00F01A0D01B06204602D501F010FD3F
:1022C0009AE701F001FD97E7142284F8702083F368
:1022D00011882B462A4629462046FFF769FE85F3DA
:1022E0001188E9E65DB1152284F8702083F3118826
:1022F00000212046D4E91D23FFF75AFEFDE60B22FC
:1023000084F8702083F311882B462A4629462046FC
:10231000FFF760FEE3E700BF744C00086C4C000858
:10232000704C000838B590F870300446002B3ED051
:10233000063BDAB20F2A34D80F2B32D8DFE803F08D
:1023400037313108223231313131313131313737A2
:10235000856FB0F886309D4214D2C3681B8AB5FBE6
:10236000F3F203FB12556DB9302383F311882B462A
:102370002A462946FFF72EFE85F311880A2384F8A2
:1023800070300EE0142384F87030302383F311880A
:10239000002320461A461946FFF70AFE002383F35E
:1023A000118838BDC36F03B198470023E7E70021C8
:1023B000204601F095FC0021204601F085FC636871
:1023C0001B6813B10621204698470623D7E7000073
:1023D00010B590F870300446142B29D017D8062B6E
:1023E00005D001D81BB110BD093B022BFBD8002141
:1023F000204601F075FC0021204601F065FC636871
:102400001B6813B1062120469847062319E0152BB7
:10241000E9D10B2380F87030302383F31188002337
:102420001A461946FFF7D6FD002383F31188DAE731
:10243000C3689B695B68002BD5D1C36F03B1984714
:10244000002384F87030CEE70023826803750369A7
:102450001B6899689142FBD25A6803604260106021
:102460005860704700238268037503691B68996888
:102470009142FBD85A680360426010605860704710
:1024800008B50846302383F311880A7D0023052A06
:1024900006D8DFE802F00B050503120E826913600F
:1024A0004FF0FF338361FFF7CFFF002383F31188E1
:1024B00008BD8269936801339360D0E900321360EC
:1024C0005A60EDE7FFF7C0BF054BD968087518687B
:1024D000026853601A600122D8600275FDF792BF4E
:1024E000C82800200C4B30B5DD684B1C87B0044673
:1024F0000FD02B46094A684600F06EF92046FFF7D8
:10250000E3FF009B13B1684600F070F9A86907B0BB
:1025100030BDFFF7D9FFF9E7C82800208124000863
:1025200038B50C4D04468161EB6881689A68914228
:1025300003D8BDE83840FFF787BF1846FFF792FF82
:1025400001230146EC6020462375BDE83840FDF7C5
:1025500059BF00BFC8280020044B1A68DB68906888
:102560009B68984294BF002001207047C828002033
:10257000084B10B51C68D868226853601A600122A5
:10258000DC602275FFF76EFF01462046BDE8104073
:10259000FDF738BFC828002038B50123084C0025B6
:1025A0002370656001F0A8FD01F0CEFD05490648E5
:1025B00001F060FE0223237085F3118838BD00BF4F
:1025C000302B00207C4C0008C828002000F044B9C3
:1025D000034A516853685B1A9842FBD8704700BFA2
:1025E000001000E08B600223086108468B82704770
:1025F0008368A3F1840243F8142C026943F8442C45
:10260000426943F8402C094A43F8242CC268A3F1DC
:10261000200043F8182C022203F80C2C002203F8A7
:102620000B2C034A43F8102C704700BF1D04000810
:10263000C828002008B5FFF7DBFFBDE80840FFF71A
:1026400041BF0000024BDB6898610F20FFF73CBFE1
:10265000C8280020302383F31188FFF7F3BF000060
:1026600008B50146302383F311880820FFF73AFFAD
:10267000002383F3118808BD064BDB6839B142683B
:1026800018605A60136043600420FFF72BBF4FF0BF
:10269000FF307047C82800200368984206D01A68A7
:1026A0000260506018469961FFF70CBF7047000048
:1026B00038B504460D462068844200D138BD036811
:1026C00023605C608561FFF7FDFEF4E7036810B5E9
:1026D0009C68A2420CD85C688A600B604C602160E8
:1026E000596099688A1A9A604FF0FF33836010BD71
:1026F000121B1B68ECE700000A2938BF0A2170B5DD
:1027000004460D460A26601901F0F0FC01F0D8FCE1
:10271000041BA54203D8751C04462E46F3E70A2E77
:1027200004D90120BDE8704001F0E4BD70BD000097
:10273000F8B5144B0D460A2A4FF00A07D96103F188
:102740001001826038BF0A22416019691446016095
:1027500048601861A81801F0B9FC01F0B1FC431BF6
:102760000646A34206D37C1C28192746354601F0AD
:10277000BDFCF2E70A2F04D90120BDE8F84001F0C2
:10278000B9BDF8BDC8280020F8B506460D4601F0D1
:1027900097FC0F4A134653F8107F9F4206D12A46F2
:1027A00001463046BDE8F840FFF7C2BFD169BB68BB
:1027B000441A2C1928BF2C46A34202D92946FFF7F8
:1027C0009BFF224631460348BDE8F840FFF77EBF35
:1027D000C8280020D8280020C0E90323002310B413
:1027E0005DF8044B4361FFF7CFBF000010B5194CF3
:1027F000236998420DD08168D0E9003213605A6095
:102800009A680A449A60002303604FF0FF33A36183
:1028100010BD0268234643F8102F53600022026067
:1028200022699A4203D1BDE8104001F059BC936877
:1028300081680B44936001F043FC2269E16992686E
:10284000441AA242E4D91144BDE81040091AFFF726
:1028500053BF00BFC82800202DE9F047DFF8BC8037
:1028600008F110072C4ED8F8105001F029FCD8F8C8
:102870001C40AA68031B9A423ED814444FF000093A
:10288000D5E90032C8F81C4013605A60C5F80090C2
:10289000D8F81030B34201D101F022FC89F311883D
:1028A000D5E9033128469847302383F311886B69B3
:1028B000002BD8D001F004FC6A69A0EB0409824621
:1028C0004A450DD2022001F015FD0022D8F8103043
:1028D000B34208D151462846BDE8F047FFF728BF6C
:1028E000121A2244F2E712EB09092946384638BF8A
:1028F0004A46FFF7EBFEB5E7D8F81030B34208D0F0
:102900001444C8F81C00211AA960BDE8F047FFF77D
:10291000F3BEBDE8F08700BFD8280020C8280020FB
:1029200000207047FEE70000704700004FF0FF30C6
:102930007047000002290CD0032904D00129074860
:1029400018BF00207047032A05D8054800EBC200D5
:102950007047044870470020704700BF544D00087E
:1029600044220020084D000870B59AB0054608467C
:10297000144601A900F0C2F801A8FEF7B7FA431CFB
:102980000022C6B25B001046C5E900342370032361
:10299000023404F8013C01ABD1B202348E4201D8BA
:1029A0001AB070BD13F8011B013204F8010C04F8D1
:1029B000021CF1E708B5302383F311880348FFF7C1
:1029C00025FA002383F3118808BD00BF382B0020AF
:1029D00090F8803003F01F02012A07D190F881207F
:1029E0000B2A03D10023C0E91D3315E003F0600377
:1029F000202B08D1B0F884302BB990F88120212AFF
:102A000003D81F2A04D8FFF7E3B9222AEBD0FAE74C
:102A1000034A426707228267C3670120704700BFED
:102A20003B22002007B5052917D8DFE801F0191669
:102A300003191920302383F31188104A01210190D2
:102A4000FFF78CFA019802210D4AFFF787FA0D482B
:102A5000FFF7A8F9002383F3118803B05DF804FBA6
:102A6000302383F311880748FFF772F9F2E7302328
:102A700083F311880348FFF789F9EBE7A84C0008B6
:102A8000CC4C0008382B002038B50C4D0C4C2A4695
:102A90000C4904F10800FFF767FF05F1CA0204F1D1
:102AA00010000949FFF760FF05F5CA7204F118002C
:102AB0000649BDE83840FFF757BF00BF104400206B
:102AC00044220020884C0008924C00089D4C0008CD
:102AD00070B5044608460D46FEF708FAC6B2204611
:102AE000013403780BB9184670BD32462946FEF70B
:102AF000E9F90028F3D10120F6E700002DE9F84FAD
:102B000005460C46FEF7F2F92C49C6B22846FFF7F7
:102B1000DFFF08B10536F6B229492846FFF7D8FF8E
:102B200008B11036F6B2632E0DD8DFF89080DFF8CA
:102B30009090244FDFF894A0DFF894B02E7846B937
:102B40002670BDE8F88F29462046BDE8F84F01F011
:102B5000B3BF252E2ED1072241462846FEF7B2F9F3
:102B600070B9DBF8003007350C3444F80C3CDBF866
:102B7000043044F8083CDBF8083044F8043CDDE756
:102B8000082249462846FEF79DF998B9A21C0E4B2B
:102B9000197802320909C95D02F8041C13F8011BF7
:102BA00001F00F015345C95D02F8031CF0D1183440
:102BB0000835C3E7013504F8016BBFE7744D000821
:102BC0009D4C0008894D000800E8F11F0CE8F11F3A
:102BD0007C4D0008BFF34F8F044B1A695107FCD19D
:102BE000D3F810215207F8D1704700BF00200052DF
:102BF00008B50D4B1B78ABB9FFF7ECFF0B4BDA6850
:102C0000D10704D50A4A5A6002F188325A60D3F8D3
:102C10000C21D20706D5064AC3F8042102F18832F6
:102C2000C3F8042108BD00BF6E46002000200052FA
:102C30002301674508B5114B1B78F3B9104B1A698E
:102C4000510703D5DA6842F04002DA60D3F8102168
:102C5000520705D5D3F80C2142F04002C3F80C21ED
:102C6000FFF7B8FF064BDA6842F00102DA60D3F8EA
:102C70000C2142F00102C3F80C2108BD6E46002071
:102C8000002000520F289ABF00F580604004002009
:102C9000704700004FF4003070470000102070476C
:102CA0000F2808B50BD8FFF7EDFF00F500330268D9
:102CB000013204D104308342F9D1012008BD002043
:102CC000FCE700000F2838B505463FD8FFF782FF24
:102CD0001F4CFFF78DFF4FF0FF3307286361C4F8E7
:102CE00014311DD82361FFF775FF030243F024035D
:102CF000E360E36843F08003E36023695A07FCD490
:102D00002846FFF767FFFFF7BDFF4FF4003100F0E3
:102D1000B3F92846FFF78EFFBDE83840FFF7C0BF84
:102D2000C4F81031FFF756FFA0F108031B0243F06F
:102D30002403C4F80C31D4F80C3143F08003C4F8F8
:102D40000C31D4F810315B07FBD4D9E7002038BD33
:102D5000002000522DE9F84F05460C46104645EA82
:102D60000203DE0602D00020BDE8F88F20F01F002D
:102D7000DFF8BCB0DFF8BCA0FFF73AFF04EB0008B7
:102D8000444503D10120FFF755FFEDE720222946F6
:102D9000204601F081FE10B920352034F0E72B46A3
:102DA00005F120021F68791CDDD104339A42F9D164
:102DB00005F178431B481C4EB3F5801F1B4B38BFF1
:102DC000184603F1F80332BFD946D1461E46FFF735
:102DD00001FF0760A5EB040C336804F11C0143F00C
:102DE00002033360231FD9F8007017F00507FAD1EA
:102DF00053F8042F8B424CF80320F4D1BFF34F8FCC
:102E0000FFF7E8FE4FF0FF332022214603602846FB
:102E1000336823F00203336001F03EFE0028BBD08C
:102E20003846B0E7142100520C2000521420005202
:102E3000102000521021005210B5084C237828B100
:102E40001BB9FFF7D5FE0123237010BD002BFCD06A
:102E50002070BDE81040FFF7EDBE00BF6E460020B9
:102E60002DE9F04F0D4685B0814658B111F00D06A1
:102E700014BF2022082211F00803019304D0431E3E
:102E800003426AD0002435E0002E37D009F11F013B
:102E900021F01F094FF00108324F05F00403DFF85D
:102EA000D0A005EA080BBBF1000F32D07869C0074B
:102EB0002FD408F101080C37B8F1060FF3D19EB9F1
:102EC000294D4946A819019201F060F904460028ED
:102ED0003AD11836019A782EF3D1494601F056F9C5
:102EE0000446002830D1019A4946204801F04EF9A5
:102EF000044668BB204605B0BDE8F08F0029C9D163
:102F000001462846029201F041F90446E0B9029ACE
:102F1000C0E713B178694107CBD5AC0702D5786912
:102F20008007C6D5019911B178690107C1D518206C
:102F3000494600FB08A0CDE9022301F027F9044629
:102F4000DDE902230028B4D04A460021204601E0F2
:102F50004A460021FDF7D2FFCCE70246002E95D16C
:102F600098E700BF9C4D0008A04600207046002056
:102F7000884600200121FFF773BF0000F8B5144D0B
:102F800001241827134E40F2FF3200210120FDF7E3
:102F9000B5FF07FB046001342A6955F80C1F01F0E6
:102FA000E1F8062CF5D137254FF4C0542046FFF741
:102FB000E1FF014628B122460748BDE8F84001F08C
:102FC000D1B8C4EBC404013D4FEAD404EED1F8BD3E
:102FD0009C4D000888460020704600200244074BA4
:102FE000D2B210B5904200D110BD441C00B253F8CB
:102FF000200041F8040BE0B2F4E700BF5040005855
:103000000E4B30B51C6F240405D41C6F1C671C6F5D
:1030100044F400441C670A4C02442368D2B243F4CF
:1030200080732360074B904200D130BD441C51F89F
:10303000045B00B243F82050E0B2F4E700440258C9
:10304000004802585040005807B5012201A900204D
:10305000FFF7C4FF019803B05DF804FB13B5044605
:10306000FFF7F2FFA04205D0012201A90020019440
:10307000FFF7C6FF02B010BD0144BFF34F8F064BF0
:10308000884204D3BFF34F8FBFF36F8F7047C3F8ED
:103090005C022030F4E700BF00ED00E0034B1A684B
:1030A0001AB9034AD2F8D0241A6070471847002092
:1030B0000040025808B5FFF7F1FF024B1868C0F353
:1030C000806008BD18470020EFF309830549683385
:1030D0004A6B22F001024A6383F30988002383F3D9
:1030E0001188704700EF00E0302080F3118862B64D
:1030F0000D4B0E4AD96821F4E0610904090C0A431A
:103100000B49DA60D3F8FC2042F08072C3F8FC204F
:10311000084AC2F8B01F116841F001011160202275
:10312000DA7783F82200704700ED00E00003FA052B
:1031300055CEACC5001000E0302310B583F31188E4
:103140000E4B5B6813F4006314D0F1EE103AEFF30A
:1031500009844FF08073683CE361094BDB6B2366A5
:1031600084F30988FFF7F8F910B1064BA36110BD8D
:10317000054BFBE783F31188F9E700BF00ED00E0A2
:1031800000EF00E02F0400083204000870B5BFF320
:103190004F8FBFF36F8F1A4A0021C2F85012BFF34E
:1031A0004F8FBFF36F8F536943F400335361BFF305
:1031B0004F8FBFF36F8FC2F88410BFF34F8FD2F8D9
:1031C000803043F6E074C3F3C900C3F34E335B01B0
:1031D00003EA0406014646EA81750139C2F86052E5
:1031E000F9D2203B13F1200FF2D1BFF34F8F536977
:1031F00043F480335361BFF34F8FBFF36F8F70BDC4
:1032000000ED00E0FEE70000214B2248224A70B5A5
:10321000904237D3214BC11EDA1C121A22F003024E
:103220008B4238BF00220021FDF768FE1C4A0023B4
:10323000C2F88430BFF34F8FD2F8803043F6E07489
:10324000C3F3C900C3F34E335B0103EA040601462E
:1032500046EA81750139C2F86C52F9D2203B13F16C
:10326000200FF2D1BFF34F8FBFF36F8FBFF34F8F9C
:10327000BFF36F8F0023C2F85032BFF34F8FBFF3FD
:103280006F8F70BD53F8041B40F8041BC0E700BFEC
:10329000C44F00080C4900200C4900200C490020B4
:1032A00000ED00E0074BD3F8D81021EA0001C3F885
:1032B000D810D3F8002122EA0002C3F80021D3F885
:1032C000003170470044025870B5D0E92443002211
:1032D0004FF0FF359E6804EB42135101D3F800090B
:1032E000002805DAD3F8000940F08040C3F800094F
:1032F000D3F8000B002805DAD3F8000B40F080402B
:10330000C3F8000B013263189642C3F80859C3F89A
:10331000085BE0D24FF00113C4F81C3870BD000008
:10332000890141F02001016103699B06FCD4122050
:10333000FFF74EB910B50A4C2046FEF7EDFD094BDC
:10334000C4F89030084BC4F89430084C2046FEF77F
:10335000E3FD074BC4F89030064BC4F8943010BD21
:103360001C47002000000840084E0008B847002015
:1033700000000440144E000870B503780546012B88
:103380005CD1434BD0F89040984258D1414B0E212C
:103390006520D3F8D82042F00062C3F8D820D3F8D3
:1033A000002142F00062C3F80021D3F80021D3F8D5
:1033B000802042F00062C3F88020D3F8802022F001
:1033C0000062C3F88020D3F88030FEF70BFA324B4E
:1033D000E360324BC4F800380023D5F89060C4F89D
:1033E000003EC02323604FF40413A3633369002B12
:1033F000FCDA01230C203361FFF7EAF83369DB07BD
:10340000FCD41220FFF7E4F83369002BFCDA002625
:103410002846A660FFF758FF6B68C4F81068DB68A1
:10342000C4F81468C4F81C6883BB1D4BA3614FF03B
:10343000FF336361A36843F00103A36070BD194BC0
:103440009842C9D1134B4FF08060D3F8D82042F096
:103450000072C3F8D820D3F8002142F00072C3F8FC
:103460000021D3F80021D3F8802042F00072C3F885
:103470008020D3F8802022F00072C3F88020D3F897
:103480008030FFF70FFF0E214D209EE7064BCDE762
:103490001C47002000440258401400400300200252
:1034A000003C30C0B8470020083C30C0F8B5D0F828
:1034B0009040054600214FF000662046FFF730FFA0
:1034C000D5F8941000234FF001128F684FF0FF30B1
:1034D000C4F83438C4F81C2804EB431201339F426B
:1034E000C2F80069C2F8006BC2F80809C2F8080BFC
:1034F000F2D20B68D5F89020C5F89830636210239B
:103500001361166916F01006FBD11220FFF760F860
:10351000D4F8003823F4FE63C4F80038A36943F4F8
:10352000402343F01003A3610923C4F81038C4F802
:1035300014380B4BEB604FF0C043C4F8103B094B01
:10354000C4F8003BC4F81069C4F80039D5F89830C5
:1035500003F1100243F48013C5F89820A362F8BD6C
:10356000E44D000840800010D0F8902090F88A10B8
:10357000D2F8003823F4FE6343EA0113C2F800389E
:10358000704700002DE9F84300EB8103D0F890501C
:103590000C468046DA680FFA81F94801166806F091
:1035A0000306731E022B05EB41134FF0000194BF7D
:1035B000B604384EC3F8101B4FF0010104F110039C
:1035C00098BF06F1805601FA03F3916998BF06F59A
:1035D000004600293AD0578A04F15801374349017F
:1035E0006F50D5F81C180B430021C5F81C382B1858
:1035F0000127C3F81019A7405369611E9BB3138AB2
:10360000928B9B08012A88BF5343D8F898209818BA
:1036100042EA034301F140022146C8F898002846D7
:1036200005EB82025360FFF77BFE08EB8900C3685D
:103630001B8A43EA845348341E4364012E51D5F853
:103640001C381F43C5F81C78BDE8F88305EB491703
:10365000D7F8001B21F40041C7F8001BD5F81C184F
:1036600021EA0303C0E704F13F030B4A2846214641
:1036700005EB83035A60FFF753FE05EB4910D0F8C2
:10368000003923F40043C0F80039D5F81C3823EA88
:103690000707D7E70080001000040002D0F894204C
:1036A0001268C0F89820FFF70FBE00005831D0F81C
:1036B000903049015B5813F4004004D013F4001F0C
:1036C0000CBF0220012070474831D0F890304901EA
:1036D0005B5813F4004004D013F4001F0CBF022009
:1036E0000120704700EB8101CB68196A0B681360F9
:1036F0004B6853607047000000EB810330B5DD6814
:10370000AA691368D36019B9402B84BF40231360A2
:103710006B8A1468D0F890201C4402EB4110013CE5
:1037200009B2B4FBF3F46343033323F0030343EA26
:10373000C44343F0C043C0F8103B2B6803F00303BD
:10374000012B0ED1D2F8083802EB411013F4807F20
:10375000D0F8003B14BF43F0805343F00053C0F84F
:10376000003B02EB4112D2F8003B43F00443C2F8A5
:10377000003B30BD2DE9F041D0F8906005460C4685
:1037800006EB4113D3F8087B3A07C3F8087B08D54A
:10379000D6F814381B0704D500EB8103DB685B689F
:1037A0009847FA071FD5D6F81438DB071BD505EB69
:1037B0008403D968CCB98B69488A5A68B2FBF0F6A1
:1037C00000FB16228AB91868DA6890420DD2121AE4
:1037D000C3E90024302383F3118821462846FFF7EC
:1037E0008BFF84F31188BDE8F081012303FA04F212
:1037F0006B8923EA02036B81CB68002BF3D021464F
:103800002846BDE8F041184700EB81034A0170B536
:10381000DD68D0F890306C692668E66056BB1A44C3
:103820004FF40020C2F810092A6802F00302012AAE
:103830000AB20ED1D3F8080803EB421410F4807FCB
:10384000D4F8000914BF40F0805040F00050C4F894
:10385000000903EB4212D2F8000940F00440C2F81C
:1038600000090122D3F8340802FA01F10143C3F838
:10387000341870BD19B9402E84BF402020602068E4
:103880001A442E8A8419013CB4FBF6F440EAC44081
:1038900040F00050C6E700002DE9F843D0F89060F2
:1038A00005460C464F0106EB4113D3F8088918F082
:1038B000010FC3F808891CD0D6F81038DB0718D5DB
:1038C00000EB8103D3F80CC0DCF81430D3F800E02F
:1038D000DA68964530D2A2EB0E024FF000091A606A
:1038E000C3F80490302383F31188FFF78DFF89F329
:1038F000118818F0800F1DD0D6F834380126A64064
:10390000334217D005EB84030134D5F89050D3F837
:103910000CC0E4B22F44DCF8142005EB0434D2F8D8
:1039200000E05168714514D3D5F8343823EA06060F
:10393000C5F83468BDE8F883012303FA01F203896E
:1039400023EA02030381DCF80830002BD1D098472A
:10395000CFE7AEEB0103BCF81000834228BF03465B
:10396000D7F8180980B2B3EB800FE3D89068A0F1C4
:10397000040959F8048FC4F80080A0EB09089844A2
:10398000B8F1040FF5D818440B4490605360C8E7B1
:103990002DE9F84FD0F8905004466E69AB691E408F
:1039A00016F480586E6103D0BDE8F84FFEF724BBD3
:1039B000002E12DAD5F8003E9B0705D0D5F8003E60
:1039C00023F00303C5F8003ED5F80438204623F061
:1039D0000103C5F80438FEF73DFB370505D5204641
:1039E000FFF772FC2046FEF723FBB0040CD5D5F898
:1039F000083813F0060FEB6823F470530CBF43F440
:103A0000105343F4A053EB6031071BD56368DB68A8
:103A10001BB9AB6923F00803AB612378052B0CD1EC
:103A2000D5F8003E9A0705D0D5F8003E23F00303F1
:103A3000C5F8003E2046FEF70DFB6368DB680BB15E
:103A400020469847F30200F1BA80B70226D5D4F891
:103A5000909000274FF0010A09EB4712D2F8003B83
:103A600003F44023B3F5802F11D1D2F8003B002B93
:103A70000DDA62890AFA07F322EA0303638104EB91
:103A80008703DB68DB6813B1394620469847013766
:103A9000D4F89430FFB29B689F42DDD9F00619D567
:103AA000D4F89000026AC2F30A1702F00F0302F47E
:103AB000F012B2F5802F00F0CA80B2F5402F09D184
:103AC00004EB8303002200F58050DB681B6A9742F9
:103AD00040F0B0803003D5F8185835D5E90303D548
:103AE00000212046FFF746FEAA0303D50121204608
:103AF000FFF740FE6B0303D502212046FFF73AFE95
:103B00002F0303D503212046FFF734FEE80203D537
:103B100004212046FFF72EFEA90203D505212046E9
:103B2000FFF728FE6A0203D506212046FFF722FE92
:103B30002B0203D507212046FFF71CFEEF0103D51A
:103B400008212046FFF716FE700340F1A780E90721
:103B500003D500212046FFF79FFEAA0703D50121C8
:103B60002046FFF799FE6B0703D502212046FFF799
:103B700093FE2F0703D503212046FFF78DFEEE06A7
:103B800003D504212046FFF787FEA80603D50521AB
:103B90002046FFF781FE690603D506212046FFF780
:103BA0007BFE2A0603D507212046FFF775FEEB05AD
:103BB00074D520460821BDE8F84FFFF76DBED4F854
:103BC00090904FF0000B4FF0010AD4F894305FFA58
:103BD0008BF79B689F423FF638AF09EB4713D3F84A
:103BE000002902F44022B2F5802F20D1D3F8002919
:103BF000002A1CDAD3F8002942F09042C3F80029C9
:103C0000D3F80029002AFBDB3946D4F89000FFF7EF
:103C100087FB22890AFA07F322EA0303238104EBD4
:103C20008703DB689B6813B13946204698470BF140
:103C3000010BCAE7910701D1D0F80080072A02F1F1
:103C400001029CBF03F8018B4FEA18283FE704EB01
:103C5000830300F58050DA68D2F818C0DCF8082039
:103C6000DCE9001CA1EB0C0C00218F4208D1DB68C1
:103C70009B699A683A449A605A683A445A6029E7BC
:103C800011F0030F01D1D0F800808C4501F1010142
:103C900084BF02F8018B4FEA1828E6E7BDE8F88FE9
:103CA00008B50348FFF774FEBDE80840FFF744BAC3
:103CB0001C47002008B50348FFF76AFEBDE808402E
:103CC000FFF73ABAB8470020D0F8903003EB411123
:103CD000D1F8003B43F40013C1F8003B70470000EB
:103CE000D0F8903003EB4111D1F8003943F40013C0
:103CF000C1F8003970470000D0F8903003EB411153
:103D0000D1F8003B23F40013C1F8003B70470000DA
:103D1000D0F8903003EB4111D1F8003923F40013AF
:103D2000C1F800397047000030B50433039C0172BC
:103D3000002104FB0325C160C0E90653049B036313
:103D4000059BC0E90000C0E90422C0E90842C0E9BF
:103D50000A11436330BD00000022416AC260C0E91D
:103D60000411C0E90A226FF00101FEF7A1BC0000B6
:103D7000D0E90432934201D1C2680AB9181D7047D4
:103D800000207047036919600021C2680132C260D7
:103D9000C269134482699342036124BF436A036189
:103DA000FEF77ABC38B504460D46E3683BB162695C
:103DB0000020131D1268A3621344E36207E0237A14
:103DC00033B929462046FEF757FC0028EDDA38BD06
:103DD0006FF00100FBE70000C368C269013BC360EC
:103DE0004369134482699342436124BF436A436138
:103DF00000238362036B03B11847704770B530230B
:103E0000044683F31188866A3EB9FFF7CBFF054667
:103E100018B186F31188284670BDA36AE26A13F8C8
:103E2000015B9342A36202D32046FFF7D5FF002334
:103E300083F31188EFE700002DE9F84F04460E46A2
:103E4000174698464FF0300989F311880025AA4695
:103E5000D4F828B0BBF1000F09D141462046FFF746
:103E6000A1FF20B18BF311882846BDE8F88FD4E973
:103E70000A12A7EB050B521A934528BF9346BBF1D4
:103E8000400F1BD9334601F1400251F8040B914217
:103E900043F8040BF9D1A36A403640354033A3629E
:103EA000D4E90A239A4202D32046FFF795FF8AF30A
:103EB0001188BD42D8D289F31188C9E730465A46E5
:103EC000FCF7F6FFA36A5E445D445B44A362E7E748
:103ED00010B5029C0433017203FB0421C460C0E9E5
:103EE00006130023C0E90A33039B0363049BC0E964
:103EF0000000C0E90422C0E90842436310BD00008D
:103F0000026A6FF00101C260426AC0E90422002225
:103F1000C0E90A22FEF7CCBBD0E904239A4201D1C2
:103F2000C26822B9184650F8043B0B607047002362
:103F30001846FAE7C3680021C2690133C3604369C8
:103F4000134482699342436124BF436A4361FEF78D
:103F5000A3BB000038B504460D46E3683BB12369B6
:103F600000201A1DA262E2691344E36207E0237A8B
:103F700033B929462046FEF77FFB0028EDDA38BD2D
:103F80006FF00100FBE7000003691960C268013AA5
:103F9000C260C269134482699342036124BF436AC9
:103FA000036100238362036B03B11847704700006D
:103FB00070B530230D460446114683F31188866A96
:103FC0002EB9FFF7C7FF10B186F3118870BDA36A41
:103FD0001D70A36AE26A01339342A36204D3E169CC
:103FE00020460439FFF7D0FF002080F31188EDE769
:103FF0002DE9F84F04460D46904699464FF0300A99
:104000008AF311880026B346A76A4FB9494620466D
:10401000FFF7A0FF20B187F311883046BDE8F88F85
:10402000D4E90A073A1AA8EB0607974228BF1746B1
:10403000402F1BD905F1400355F8042B9D4240F851
:10404000042BF9D1A36A40364033A362D4E90A2392
:104050009A4204D3E16920460439FFF795FF8BF3B8
:1040600011884645D9D28AF31188CDE729463A46C8
:10407000FCF71EFFA36A3D443E443B44A362E5E7D0
:10408000D0E904239A4217D1C3689BB1836A8BB1EC
:10409000043B9B1A0ED01360C368013BC360C36925
:1040A0001A4483699A42026124BF436A0361002370
:1040B00083620123184670470023FBE700F01EBA15
:1040C000014B586A704700BF000C0040034B0022B0
:1040D00058631A610222DA60704700BF000C00408A
:1040E000014B0022DA607047000C0040014B58631E
:1040F000704700BF000C0040024B034A1A60034A9D
:104100005A6070476C4800201049002000000220CF
:10411000074B494210B55C68201A08401968821A9A
:104120008A4203D3A24201D85A6010BD0020FCE7A6
:104130006C48002008B5302383F31188FFF7E8FFAF
:10414000002383F3118808BD04480121044B036058
:104150000023C0E901330C3000F0D4B874480020CB
:1041600035410008CB1D083A23F00703591A521AAB
:10417000012110B4D2080024C0E9004384600C304F
:104180001C605A605DF8044B00F0BCB82DE9F84F94
:10419000364ECD1D0F46002818BF0646082A4FEAA6
:1041A000D50538BF082206F10C08341D914640465B
:1041B00000F0C4F809F10701C9F1000E2246246895
:1041C0006CB9404600F0C4F83368CBB308224946C6
:1041D000E8009847044698B340E9026730E004EBF2
:1041E000010CD4F804A00CEA0E0C0AF10100ACF1A9
:1041F000080304EBC0009842E0D9A0EB0C0CB5EB2F
:10420000EC0F4FEAEC0BD9D89C421CD204F1080207
:10421000AB45A3EB02024FEAE202626009D9691CD6
:10422000ED43206803EBC1025D44556043F8310063
:1042300022601C465F60404644F8086B00F088F836
:104240002046BDE8F88FAA45216802D111602346B7
:10425000EFE7013504EBC50344F8351003F108011D
:10426000401AC01058601360F1E700BF7448002086
:10427000FEE7000070B51B4B0025044686B0586071
:104280000E4685620163FEF72FFF04F11003A5605F
:10429000E562C4E904334FF0FF33C4E90044C4E9E4
:1042A0000635FFF70DFF2B46024604F13401204688
:1042B000C4E9082380230C4A2565FEF793F90123FE
:1042C0000A4AE06000920375684672680192B2681B
:1042D000CDE90223064BCDE90435FEF7ABF906B074
:1042E00070BD00BF302B0020204E0008254E000876
:1042F00071420008024AD36A1843D062704700BF77
:10430000C8280020C0E90000816070478368013B35
:10431000002B10B583600CDA074BDC684368A061A2
:10432000206063601C6044600520FEF7CDF8A06942
:1043300010BD0020FCE700BFC828002008B53023CE
:1043400083F31188FFF7E2FF002383F3118808BD90
:1043500008B5302383F3118883680133002B836011
:1043600007DC036800211A68026050601846FEF7F7
:10437000D7F8002383F3118808BD00004B68436021
:104380008B688360CB68C3600B6943614B690362D0
:104390008B6943620B6803607047000008B53C4BB3
:1043A00040F2FF713B48D3F888200A43C3F88820C5
:1043B000D3F8882022F4FF6222F00702C3F8882095
:1043C000D3F88820D3F8E0200A43C3F8E020D3F8DC
:1043D00008210A43C3F808212F4AD3F808311146AF
:1043E000FFF7CCFF00F5806002F11C01FFF7C6FF6C
:1043F00000F5806002F13801FFF7C0FF00F5806032
:1044000002F15401FFF7BAFF00F5806002F170017C
:10441000FFF7B4FF00F5806002F18C01FFF7AEFFFB
:1044200000F5806002F1A801FFF7A8FF00F58060A9
:1044300002F1C401FFF7A2FF00F5806002F1E00184
:10444000FFF79CFF00F5806002F1FC01FFF796FF8B
:1044500002F58C7100F58060FFF790FF00F01AF90B
:104460000E4BD3F8902242F00102C3F89022D3F809
:10447000942242F00102C3F894220522C3F8982046
:104480004FF06052C3F89C20054AC3F8A02008BD35
:1044900000440258000002582C4E000800ED00E0D5
:1044A0001F00080308B500F0D7FAFEF775F8104BA7
:1044B000D3F8DC2042F04002C3F8DC20D3F804211A
:1044C00022F04002C3F80421D3F80431094B1A68E2
:1044D00042F008021A601A6842F004021A60FEF7FD
:1044E000DDFDFEF74BFDBDE80840FEF7CDBA00BF8D
:1044F000004402580018024870470000114BD3F8DE
:10450000E82042F00802C3F8E820D3F8102142F076
:104510000802C3F810210C4AD3F81031D36B43F0D2
:104520000803D363C722094B9A624FF0FF32DA6265
:1045300000229A615A63DA605A6001225A611A6055
:10454000704700BF004402580010005C000C00409F
:10455000094A08B51169D3680B40D9B29B076FEAC5
:104560000101116107D5302383F31188FEF72EF87E
:10457000002383F3118808BD000C0040064BD3F8DC
:10458000DC200243C3F8DC20D3F804211043C3F835
:104590000401D3F8043170470044025808B53C4B7D
:1045A0004FF0FF31D3F8802062F00042C3F8802042
:1045B000D3F8802002F00042C3F88020D3F8802096
:1045C000D3F88420C3F88410D3F884200022C3F8E1
:1045D0008420D3F88400D86F40F0FF4040F4FF00FF
:1045E00040F4DF4040F07F00D867D86F20F0FF40F4
:1045F00020F4FF0020F4DF4020F07F00D867D86F60
:10460000D3F888006FEA40506FEA5050C3F8880032
:10461000D3F88800C0F30A00C3F88800D3F88800F4
:10462000D3F89000C3F89010D3F89000C3F890200E
:10463000D3F89000D3F89400C3F89410D3F8940002
:10464000C3F89420D3F89400D3F89800C3F89810D6
:10465000D3F89800C3F89820D3F89800D3F88C00CA
:10466000C3F88C10D3F88C00C3F88C20D3F88C00DE
:10467000D3F89C00C3F89C10D3F89C10C3F89C207E
:10468000D3F89C30FCF7C0FEBDE8084000F0B8B994
:104690000044025808B50122534BC3F80821534B7C
:1046A000D3F8F42042F00202C3F8F420D3F81C211E
:1046B00042F00202C3F81C210222D3F81C314C4BF9
:1046C000DA605A689104FCD54A4A1A6001229A605D
:1046D000494ADA6000221A614FF440429A61444B21
:1046E0009A699204FCD51A6842F480721A603F4BB2
:1046F0001A6F12F4407F04D04FF480321A67002200
:104700001A671A6842F001021A60384B1A6850079B
:10471000FCD500221A611A6912F03802FBD101217E
:1047200019604FF0804159605A67344ADA62344A5E
:104730001A611A6842F480321A602C4B1A6891038D
:10474000FCD51A6842F480521A601A689204FCD5AB
:104750002C4A2D499A6200225A63196301F57C01A3
:10476000DA6301F2E71199635A64284A1A64284A05
:10477000DA621A6842F0A8521A601C4B1A6802F0FA
:104780002852B2F1285FF9D148229A614FF4886229
:10479000DA6140221A621F4ADA641F4A1A651F4A08
:1047A0005A651F4A9A6532231E4A1360136803F044
:1047B0000F03022BFAD10D4A136943F0030313616F
:1047C000136903F03803182BFAD14FF00050FFF7AC
:1047D000D5FE4FF08040FFF7D1FE4FF00040BDE81E
:1047E0000840FFF7CBBE00BF0080005100440258D4
:1047F0000048025800C000F0020000010000FF0164
:10480000008890081210200063020901470E050875
:10481000DD0BBF0120000020000001100910E000A6
:1048200000010110002000524FF0B04208B5D2F84C
:10483000883003F00103C2F8883023B1044A1368BA
:104840000BB150689847BDE80840FEF775BC00BF43
:104850008C4800204FF0B04208B5D2F8883003F001
:104860000203C2F8883023B1044A93680BB1D068C0
:104870009847BDE80840FEF75FBC00BF8C480020A9
:104880004FF0B04208B5D2F8883003F00403C2F804
:10489000883023B1044A13690BB150699847BDE8C9
:1048A0000840FEF749BC00BF8C4800204FF0B042E2
:1048B00008B5D2F8883003F00803C2F8883023B175
:1048C000044A93690BB1D0699847BDE80840FEF7E8
:1048D00033BC00BF8C4800204FF0B04208B5D2F87E
:1048E000883003F01003C2F8883023B1044A136AF9
:1048F0000BB1506A9847BDE80840FEF71DBC00BFE9
:104900008C4800204FF0B04310B5D3F8884004F431
:104910007872C3F88820A30604D5124A936A0BB1B3
:10492000D06A9847600604D50E4A136B0BB1506BE2
:104930009847210604D50B4A936B0BB1D06B98476F
:10494000E20504D5074A136C0BB1506C9847A305D8
:1049500004D5044A936C0BB1D06C9847BDE8104065
:10496000FEF7EABB8C4800204FF0B04310B5D3F8F7
:10497000884004F47C42C3F88820620504D5164AB6
:10498000136D0BB1506D9847230504D5124A936DF2
:104990000BB1D06D9847E00404D50F4A136E0BB1EC
:1049A000506E9847A10404D50B4A936E0BB1D06E9C
:1049B0009847620404D5084A136F0BB1506F9847AB
:1049C000230404D5044A936F0BB1D06F9847BDE818
:1049D0001040FEF7B1BB00BF8C48002008B503486B
:1049E000FCF77AFEBDE80840FEF7A6BB5C24002079
:1049F00008B5FFF7ADFDBDE80840FEF79DBB000020
:104A0000062108B50846FCF7EDFE06210720FCF755
:104A1000E9FE06210820FCF7E5FE06210920FCF747
:104A2000E1FE06210A20FCF7DDFE06211720FCF737
:104A3000D9FE06212820FCF7D5FE09217A20FCF7B3
:104A4000D1FE07213220FCF7CDFE0C212520BDE848
:104A50000840FCF7C7BE000008B5FFF79FFD00F057
:104A60000DF8FDF77DF8FDF755FAFDF727F9FFF78B
:104A700043FDBDE80840FFF721BB00000023054AC5
:104A800019460133102BC2E9001102F10802F8D1D6
:104A9000704700BF8C48002010B501390244904295
:104AA00001D1002005E0037811F8014FA34201D0A5
:104AB000181B10BD0130F2E7034611F8012B03F873
:104AC000012B002AF9D1704753544D333248373FF8
:104AD0003F3F0053544D3332483733782F373278C5
:104AE0000053544D3332483734332F3735332F3753
:104AF0003530000001105A00031059000120580001
:104B00000320560010000240080002400008024046
:104B100000000B0028000240080002400408024088
:104B200006010C0040000240080002400808024054
:104B300010020D0058000240080002400C0802401C
:104B400016030E00700002400C00024010080240E4
:104B500000040F00880002400C00024014080240CC
:104B600006051000A00002400C0002401808024098
:104B700010061100B80002400C0002401C08024060
:104B800016072F00100402400804024020080240CB
:104B900000083800280402400804024024080240AB
:104BA0000609390040040240080402402808024077
:104BB000100A3A0058040240080402402C0802403F
:104BC000160B3B00700402400C0402403008024007
:104BD000000C3C00880402400C04024034080240EF
:104BE000060D4400A00402400C04024038080240B4
:104BF000100E4500B80402400C0402403C0802407C
:104C0000160F4600009600000000000000000000A3
:104C10000000000000000000000000000000000094
:104C2000211B00080D1B0008491B0008351B00084C
:104C3000411B00082D1B0008191B0008051B00085C
:104C4000551B000800000000391C0008251C000846
:104C5000611C00084D1C0008591C0008451C000878
:104C6000311C00081D1C00086D1C0008000000001D
:104C7000010000000000000063300000784C0008D4
:104C800020290020302B00204172647550696C6F20
:104C9000740025424F415244252D424C0025534576
:104CA0005249414C250000000200000000000000B5
:104CB000591E0008C91E000840004000E0430020C3
:104CC000F04300200200000000000000030000008C
:104CD00000000000111F000800000000100000008C
:104CE000004400200000000001000000000000005F
:104CF0001C47002001010200252A00083529000870
:104D0000D1290008B529000843000000104D000813
:104D100009024300020100C032090400000102023E
:104D200001000524001001052401000104240202F1
:104D30000524060001070582030800FF090401009D
:104D4000020A000000070501024000000705810279
:104D500040000000120000005C4D0008120110012C
:104D60000200004009124157000201020301000045
:104D70000403090425424F41524425004D69636FE5
:104D8000416972373433763200303132333435365C
:104D900037383941424344454600000000000020B6
:104DA00000000200020000000000003000000400CB
:104DB00008000000000000240000080004000000BB
:104DC0000004000000FC00000200000000000430AD
:104DD0000080000008000000000000380000010012
:104DE00001000000000000006D20000825230008DD
:104DF000D1230008400040005448002054480020BF
:104E00000100000064480020800000004001000014
:104E10000800000000010000001000000800000071
:104E20006D61696E0069646C650000000000A86A2D
:104E300000000000AAAAAAAA00001464FFFF000054
:104E40000000000070A70A00000000010000000040
:104E5000AAAAAAAA00000001FFFF000000000000AB
:104E6000000000000000000000000000AAAAAAAA9A
:104E700000000000FFFF0000000000000000000034
:104E80000005000000000000AAAAAAAA0005000070
:104E9000FFFF000000000000000000001001000003
:104EA00000000000AAAAAAAA00000000EBFF000070
:104EB00000000000000000000000000000000000F2
:104EC000AAAAAAAA00000000FFFF0000000000003C
:104ED000000000000000000000000000AAAAAAAA2A
:104EE00000000000FFFF00000000000000000000C4
:104EF0000000000000000000AAAAAAAA000000000A
:104F0000FFFF0000000000000000000000000000A3
:104F100000000000AAAAAAAA00000000FFFF0000EB
:104F20000000000000000000000000000000000081
:104F3000AAAAAAAA00000000FFFF000000000000CB
:104F4000000000000000000000000000AAAAAAAAB9
:104F500000000000FFFF0000000000000000000053
:104F60009B0400000000000000001A000000000088
:104F7000FF000000382B00205C240020000000000F
:104F8000C84A000883040000D34A00085004000007
:104F9000E14A0008009600000000080096000000AA
:104FA0000008000004000000704D00080000000030
:104FB00000000000000000000000000000000000F1
:044FC00000000000ED
:00000001FF
